:1000000012C02AC029C028C027C026C025C024C0CD
:1000100023C022C021C020C01FC01EC01DC01CC0E4
:100020001BC01AC019C011241FBECFEDCDBF10E0F8
:10003000A0E6B0E0EAE8F0E003C0C89531960D9282
:10004000A036B107D1F710E0A0E6B0E001C01D92E4
:10005000A036B107E1F70AC0D3CF80E593ECA0E06A
:10006000B0E0C297A109B109E1F70895CFEDD0E062
:10007000DEBFCDBF8FEF87BB8FE088BBC0E0EDDF79
:0A008000C8BBCE5FCF3FD9F7F9CF20
:00000001FF
